:100000000C94AA010C94D2010C94D2010C94D2014C
:100010000C94D2010C94D2010C94D2010C94D20114
:100020000C94D2010C9472120C94D2010C94D20153
:100030000C94D2010C94030C0C94D2010C94D201B8
:100040000C94D2010C94D2010C94D2010C94D201E4
:100050000C94D2010C94D2010C94D2010C94D201D4
:100060000C94D2010C94D20154095A095D0960091B
:100070006309660969096C096F09720975097809CC
:1000800020506F6C6F6C750033F720526F626F7485
:100090000044656D6F0050726F6772616D0055733B
:1000A00065204220746F0073656C6563742E005088
:1000B000726573732042002D747279206974210077
:1000C000205468616E6B20002020796F752100201C
:1000D000204D61696E0020204D656E75004261748F
:1000E00074657279004C454473004C434400536579
:1000F0006E736F7273004D6F746F7273004D757312
:100100006963005472696D706F740054696D657233
:10011000007F4120A54220437E000642003E673317
:10012000323E3E633332003E3E6333323E6733320B
:1001300000216333320021653332002167333200FE
:100140002176383E3E63333200000000000000009C
:100150001F1F1F1F1F1F1F04060505041C1C000076
:10016000020105091E08042120543132304F354C5C
:10017000313661676166616561206461632B61642A
:100180006165612066613C61613C6261632361205D
:1001900064616323616461656120664F36646364F2
:1001A0003C622D643C61643C6720643C662B643C8B
:1001B00067643C61643C622D20643C64643C65641B
:1001C0003C662B643C6720643C662B643C67643C63
:1001D00061644C384D533C622D643C622D64204D6B
:1001E0004C652D3C67652D3C67204D53633C616336
:1001F0003C61204D4C643C66643C66204F354D5359
:10020000622D67622D674D4C3E6323653E63236517
:10021000204D532061666166204D4C206763236743
:100220006323204D532066646664204D4C20653C5A
:10023000622D653C622D4F364C31367261676166C6
:100240006165612064616323616461656120666149
:100250003C61613C6261632361206461632361648A
:100260006165612066616561646163613C622D6105
:10027000636164673C622D67206567646763673C00
:10028000622D67203C61673C622D6763663C616656
:1002900020646663663C622D663C61663C67663C32
:1002A00061663C622D653C6765206323653C622D79
:1002B000653C61653C6765203C66653C67653C6103
:1002C000643C66644F35653E65653E65663E6466C2
:1002D0003E6420622D3E6323622D3E6323613E64B3
:1002E000663E6420653E65653E65663E64663E64C6
:1002F000653E643E63233E64623E643E6323622047
:100300003E63236167616567666520664F36646397
:100310002364666463233C6220632334002020202E
:10032000202020200720467567756520696E2044CF
:10033000204D696E6F72202D206279204A2E532E37
:100340002042616368200720202020202020000018
:10035000600F610F11241FBECFEFD4E0DEBFCDBF11
:1003600011E0A0E0B1E0E4EFF7E202C005900D92E9
:10037000A836B107D9F711E0A8E6B1E001C01D9297
:10038000A93CB107E1F713E0C2E5D3E004C022972E
:10039000FE010E94E913C035D107C9F70E94BC06CF
:1003A0000C94ED130C9400001F9382E30E94D90C6F
:1003B000182F81FF03C081E391E007C084FF03C0D1
:1003C00086E391E002C08BE391E00E94F00B812F65
:1003D0000E949F0C812F1F910895EF92FF920F931F
:1003E0001F938C017B010E94EB0DC8010E94860EB9
:1003F00061E070E080E090E00E94D80DC7010E94AB
:10040000860E88EE93E00E94B1121F910F91FF902B
:10041000EF9008951F93CF93DF9366ED70E08FEC1C
:1004200090E00E94ED01C6E0D0E00E94EB0D61E09B
:1004300070E080E090E00E94D80D81E191E00E94A0
:10044000860E60E070E080E090E00E94D80DE091C0
:100450006C01F0916D01EE0FFF1FEE5CFE4F80818D
:1004600091810E94860E81E00E94B50D82E30E9478
:10047000520C8823D9F782E30E94D90C182F81FFF0
:100480000AC081E391E00E94F00B80916C01909191
:100490006D01019758C084FF4BC00E94AA0D0E94B5
:1004A000EB0D86E391E00E94F00B812F0E949F0CE0
:1004B0001CC061E070E080E090E00E94D80D8AE10D
:1004C00091E00E94860E60E070E080E090E00E9483
:1004D000D80DE0916C01F0916D01EE0FFF1FEC5D06
:1004E000FE4F0190F081E02D099580E10E94520CB1
:1004F0008823F9F260E070E080E090E00E9431082B
:100500000E944208109269011092680110926B01DA
:1005100010926A0180E00E94CB0E80E00E94D20E11
:1005200086E391E00E94F00BDF91CF911F91089537
:1005300085FF0DC08BE391E00E94F00B80916C0170
:1005400090916D01019690936D0180936C01809163
:100550006C0190916D0197FF04C0D0936D01C09321
:100560006C0180916C0190916D0107970CF45DCF47
:1005700010926D0110926C0158CFCF93DF93C0E0C1
:10058000D0E08AE090E00E94B11280E10E94520C1B
:10059000882311F081E005C02196C931D10589F782
:1005A00080E0DF91CF910895EF92FF920F931F9318
:1005B0000E9406137B018C01809171019091720160
:1005C000A0917301B09174010097A105B10501F1EB
:1005D0008091790190917A01A0917B01B0917C0189
:1005E0002091750130917601409177015091780109
:1005F000821B930BA40BB50B8E0D9F1DA01FB11F6B
:100600008093790190937A01A0937B01B0937C0150
:10061000E0927501F09276010093770110937801D2
:1006200082E00E94520C8823F9F0809170018823A7
:10063000D9F481E0809370011092710110927201DF
:1006400010927301109274011092790110927A0144
:1006500010927B0110927C010E943408882321F4BF
:1006600081E391E00E94F00B82E00E94520C88230B
:1006700011F41092700180E20E94520C882339F12B
:1006800080916F01882319F581E080936F0120E04C
:1006900030E040E050E08091710190917201A091B2
:1006A0007301B09174010097A105B10521F421E017
:1006B00030E040E050E020937101309372014093AC
:1006C0007301509374018BE391E00E94F00B80E280
:1006D0000E94520C882311F410926F0160917901ED
:1006E00070917A0180917B0190917C0120EC37E23E
:1006F00049E050E00E949513CA01B9012AE030E0B8
:1007000040E050E00E9495130E94740E60917901C0
:1007100070917A0180917B0190917C0120E63AEE04
:1007200040E050E00E949513CA01B9012AE030E090
:1007300040E050E00E9495130E94740E8AE30E94EC
:100740009E0E6091790170917A0180917B01909168
:100750007C0128EE33E040E050E00E949513CA018E
:10076000B9012CE330E040E050E00E9495132AE00C
:1007700030E040E050E00E949513CA01B9010E94A8
:10078000740E6091790170917A0180917B01909152
:100790007C0128EE33E040E050E00E949513CA014E
:1007A000B9012CE330E040E050E00E9495132AE0CC
:1007B00030E040E050E00E949513162F70E080E09A
:1007C00090E00E94740E8EE20E949E0E609179016C
:1007D00070917A0180917B0190917C0124E630E058
:1007E00040E050E00E949513CA01B9012AE030E0D0
:1007F00040E050E00E9495130E94740E60917901D0
:1008000070917A0180917B0190917C012AE030E027
:1008100040E050E00E949513CA01B9012AE030E09F
:1008200040E050E00E9495130E94740E80916E018A
:100830001817A1F08091790190917A01A0917B0124
:10084000B0917C010097A105B10541F00E943408E8
:10085000882321F480E491E00E94F00B10936E0154
:100860001F910F91FF90EF900895CF93DF930E9417
:10087000061320917D0130917E0140917F015091BE
:100880008001621B730B840B950B6B3F7105810517
:10089000910530F1C0E0D0E080918101FE01E80FC8
:1008A000F11DE35EFC4FE4918E2F0E949E0E219677
:1008B000C830D10589F70E94061360937D017093BB
:1008C0007E0180937F0190938001809181018F5FF1
:1008D0008093810190E00896C29710F010928101F8
:1008E0000E943408882321F487E691E00E94F00BEF
:1008F00084E690E00E94B112DF91CF9108950F93AA
:100900001F9382E00E94520C20916801309169018E
:100910008823E9F0232B89F488EC90E00E94B1123F
:1009200082E00E94520C882341F490E08091830180
:10093000882309F491E0909383018091680190915C
:1009400069010A96909369018093680106C0245159
:100950003040309369012093680180E20E94520C7C
:1009600020916A0130916B018823E9F0232B89F4EF
:1009700088EC90E00E94B11280E20E94520C882321
:1009800041F490E080918201882309F491E09093F2
:10099000820180916A0190916B010A9690936B019C
:1009A00080936A0106C02451304030936B0120933C
:1009B0006A01809168019091690197FF04C01092CB
:1009C00069011092680180916801909169018F3FDF
:1009D000910539F034F08FEF90E0909369018093A6
:1009E000680180916A0190916B0197FF04C0109299
:1009F0006B0110926A0180916A0190916B018F3FA7
:100A0000910539F034F08FEF90E090936B01809373
:100A10006A0180916801909169016AE170E00E9429
:100A20006013FB01EF5BFE4F108180916A01909192
:100A30006B016AE170E00E946013FB01EF5BFE4F07
:100A40000081812F0E949E0E80918301882311F4E2
:100A500081E401C081E60E949E0E812F0E949E0EBD
:100A600060E070E085E090E00E94D80D802F0E9449
:100A70009E0E80918201882311F483E401C083E6F5
:100A80000E949E0E802F0E949E0EA0916A01B0913E
:100A90006B0180918201882319F441E050E002C08B
:100AA0004FEF5FEFE0916801F09169018091830160
:100AB000882319F421E030E002C02FEF3FEF4A9F76
:100AC000B0014B9F700D5A9F700D11242E9FC001D5
:100AD0002F9F900D3E9F900D11240E94310882E3BC
:100AE00090E00E94B1121F910F910895EF92FF9232
:100AF0000F93DF93CF9300D0CDB7DEB70E940613DC
:100B0000F62E80E00E94D90E0E94430FA0E0B0E0D4
:100B1000BC01CD010E94740E80E091E00E94970E0E
:100B20002AE0E22E1CC00E94430F9A8389834FE083
:100B300068EC70E00E9423090E9DC00111242981F8
:100B40003A81281739072CF480E00E94CB0E81E00F
:100B500004C081E00E94CB0E80E00E94D20E0E9471
:100B60000613062F0F190436F0F20F900F90CF9155
:100B7000DF910F91FF90EF900895EF92FF920F9306
:100B80001F93DF93CF93CDB7DEB72A970FB6F894B4
:100B9000DEBF0FBECDBF80E20E94520C9E012F5FD0
:100BA0003F4F882311F060E001C061E0C9010E945D
:100BB000660F8E010F5F1F4F3BE0E32EF12CEC0E12
:100BC000FD1EF801819191918F0169EC70E00E9406
:100BD0004C13FB01EF5BFE4F80810E949E0E0E15B1
:100BE0001F0579F780E20E94520C882319F084E0F7
:100BF00091E002C088E091E00E94970E84E690E0C8
:100C00000E94B1122A960FB6F894DEBF0FBECDBF78
:100C1000CF91DF911F910F91FF90EF9008958CE09D
:100C200091E00E94000C80E191E00E94970E81E02B
:100C30000E94CB0E0E94BD028823F9F40E94CB0EC5
:100C40000E94BD028823C9F486E191E00E94000C55
:100C500060E070E080E090E00E94D80D8BE191E0D0
:100C60000E94970E81E00E94D20E0E94BD0288234E
:100C700021F40E94D20E0E94BD0208950E945D0FD1
:100C8000AA2797FDA095BA2FBC01CD010E94740E32
:100C900081E291E00E94970E84E690E00E94B112FA
:100CA00008950F931F9309E411E060E0C8010E94CA
:100CB000C80E61E0C80101960E94C80E62E0C8013A
:100CC00002960E94C80E63E0C80104960E94C80EF6
:100CD00064E0C80105960E94C80E65E0C80106964A
:100CE0000E94C80E66E08FE591E00E94C80E67E0A2
:100CF00087E591E00E94C80E0E94EB0D1F910F91B5
:100D0000089580ED97E00E94970F0E9451068DE1B3
:100D100091E00E94F00B68E870E080E890E00E94AB
:100D2000ED0166E970E081E990E00E94ED0167EA7B
:100D300070E08EE990E00E94ED010E94EB0D8FEAD9
:100D400090E00E94860E61E070E080E090E00E94FA
:100D5000D80D87EB90E00E94860E0E94D40184FF9C
:100D6000FCCF87E291E00E94F00B68EC70E080EC31
:100D700090E00E94ED0108950E9481060E940A02FF
:100D8000FDCFCF93DF93BC018230910510F462E078
:100D900070E0A091C701B091C801ED01E0E0F0E082
:100DA00040E050E021C0888199818617970769F457
:100DB0008A819B81309719F09383828304C090933A
:100DC000C8018093C701FE0134C06817790738F461
:100DD0004115510519F08417950708F4AC01FE017F
:100DE0008A819B819C01E9012097E9F64115510513
:100DF000A9F1CA01861B970B049708F4BA01E0E039
:100E0000F0E02AC08D919C91119784179507F9F411
:100E10006417750781F412968D919C911397309702
:100E200019F09383828304C09093C8018093C70113
:100E3000FD0132964CC0CA01861B970BFD01E80FDD
:100E4000F91F6193719302978D939C9340C0FD01AC
:100E5000828193819C01D9011097A1F68091C501EF
:100E60009091C601892B41F48091640190916501B4
:100E70009093C6018093C50140916601509167012E
:100E80004115510541F44DB75EB7809162019091D3
:100E90006301481B590B2091C5013091C601CA015D
:100EA000821B930B8617970780F0AB014E5F5F4F55
:100EB0008417950750F0420F531F5093C60140937B
:100EC000C501F9016193719302C0E0E0F0E0CF0148
:100ED000DF91CF910895CF93DF93009709F450C02D
:100EE000EC0122971B821A82A091C701B091C80120
:100EF000109709F140E050E0AC17BD0708F1BB8343
:100F0000AA83FE0121913191E20FF31FAE17BF07B3
:100F100079F48D919C911197280F391F2E5F3F4FC7
:100F20003983288312968D919C9113979B838A8392
:100F30004115510571F4D093C801C093C70120C079
:100F400012968D919C911397AD01009711F0DC01E1
:100F5000D3CFFA01D383C28321913191E20FF31FE2
:100F6000CE17DF0769F488819981280F391F2E5F1A
:100F70003F4FFA01318320838A819B81938382834F
:100F8000DF91CF910895809184018823F1F481E06D
:100F90008093840183EF8093B0008091B00084BD82
:100FA00082E08093B1008091B10085BD1092B400C1
:100FB0008091B4008093B3008091B30088BD88B560
:100FC00087BD8AB188668AB9239A0895CF93DF9343
:100FD000EC010E94C307D7FD02C020E004C0D095F9
:100FE000C195DF4F21E0CE01CF3FD10519F014F0BC
:100FF0008FEF90E0222319F018BC87BD02C088BD96
:1010000017BCDF91CF910895CF93DF93EC010E943D
:10101000C307D7FD02C020E004C0D095C195DF4FC3
:1010200021E0CE01CF3FD10519F014F08FEF90E011
:10103000222329F01092B4008093B30004C080935F
:10104000B4001092B300DF91CF9108950F931F93D6
:101050008B010E94E607C8010E9404081F910F91AE
:1010600008950E942608089580914B01882339F045
:1010700020E08091860190918701892B09F021E081
:10108000822F089510926F00E1E8F0E08081887F60
:101090008160808380E29EE4909389008093880041
:1010A00010928B0010928A00229881E080934B016D
:1010B00010928701109286010895A0E0B0E0E3E667
:1010C000F8E00C94B813FC015B01C42E80918501FB
:1010D0008823C1F481E08093850110926F002298EB
:1010E00083E28093800089E18093810010928200E6
:1010F00080E29EE4909389008093880010928B0098
:1011000010928A0010924B01F7FD03C0DD24D394A6
:1011100003C0FF779AE0D92E80918100082F10E05C
:10112000087F10702D2D30E080E991E0AC01249F04
:10113000C001259F900D349F900D11248E179F079D
:1011400098F4EF0157E2E131F50710F0C0E1D7E282
:101150009E0140E050E060E07DE281E391E00E948A
:101160007313790101601DC088E2D89E802D11247F
:10117000C82FD0E0CE17DF0708F4EF019E0140E052
:1011800050E08AE0D81629F460E478E78DE791E032
:1011900004C060EA75E286E290E00E947313790170
:1011A00002604AE0D41639F4CE0105966AE070E098
:1011B0000E944C13EB0153E0C83ED50711F4B50172
:1011C0000FC0BE0180E090E0950140E050E00E9439
:1011D000211328EE33E040E050E00E949513B9015E
:1011E000CC2011F4229806C0229A8FE08C1510F4BE
:1011F0008FE0C82E10926F0000938100F09289005A
:10120000E0928800209188003091890080E190E090
:101210008C19910902C0369527958A95E2F730938B
:101220008B0020938A0070938D0160938C0186B3AC
:101230008FEF86BB81E080936F007894CDB7DEB7E7
:10124000EAE00C94D4130E945D080895CF93DF93D5
:10125000EB018F3F11F0442329F440E0BE0188EEFA
:1012600093E067C0813110F420E005C0282F2051A1
:10127000203608F02FE5822F6CE00E944013382FB3
:10128000682F70E084EF9FEF689FF001699FF00D79
:10129000789FF00D1124E20FF11DEC30F10538F4C8
:1012A000EC5CFF4F0C94E7138CE991E023C080E0E5
:1012B00090E020C085EB91E01DC08FEC91E01AC05A
:1012C0008AEE91E017C087E092E014C086E292E0D7
:1012D00011C087E492E00EC089E692E00BC08EE870
:1012E00092E008C085EB92E005C08EED92E002C06E
:1012F0008AE093E0373071F002C0880F991F6A9539
:10130000E2F7323020F005966AE070E00BC08050C2
:1013100090480BC026E0880F991F2A95E1F70296A6
:1013200065E070E00E944C13CB01403108F04FE0C3
:10133000BE010E945D08DF91CF91089520918B013D
:10134000E0918601F0918701222311F0949101C070
:101350009081892F81548A3108F4905E903221F473
:101360003196E130F10581F7F0938701E093860132
:10137000892F0895CF93DF930E949E09282FC0E004
:10138000D0E01DC0CE0143E0880F991F4A95E1F7D8
:10139000CC0FDD1FC80FD91F822F992787FD90958D
:1013A000C80FD91FE097809186019091870101961F
:1013B00090938701809386010E949E09282F822F97
:1013C00080538A30F8F2CE01DF91CF910895A0E0EA
:1013D000B0E0EDEEF9E00C94B61380904C01B090C3
:1013E0008901BB2021F060918A01662399F4A090C5
:1013F0008A010091510110915201E0904D01F0904D
:101400004E01C0914F01D0915001C0905301D09036
:10141000540108C140E070E08FEF0E94260910924D
:101420008A01CBC114E0812EBB2404EF11E0B4E0AB
:10143000EB2EF12CC0EDD7E0A4E09A2EFFE0CF2EEA
:10144000D12C0E949E09282F8091860190918701BE
:1014500001969093870180938601263609F498C0FF
:101460002736CCF42236A1F1233674F42E3361F101
:101470002F3334F42132B1F22C3309F00BC126C0E2
:10148000213609F007C121C1243609F451C025369F
:101490000CF066C035C02F3609F4C1C0203754F4B3
:1014A0002C3609F4A5C02D3609F4A6C0273609F05C
:1014B000F1C086C0243709F4D1C0263709F4E6C04C
:1014C000223709F0E7C0B0C08394BBCF8A94B9CF6C
:1014D000A0928A01B09289011093520100935101A8
:1014E000F0924E01E0924D01D0935001C0934F0114
:1014F00090924C01D0925401C09253012BE0FCC059
:10150000A0928A01B0928901109352010093510177
:10151000F0924E01E0924D01D0935001C0934F01E3
:1015200090924C01D0925401C092530120E0E4C04B
:10153000A0928A01B0928901109352010093510147
:10154000F0924E01E0924D01D0935001C0934F01B3
:1015500090924C01D0925401C092530122E0CCC031
:10156000A0928A01B0928901109352010093510117
:10157000F0924E01E0924D01D0935001C0934F0183
:1015800090924C01D0925401C092530124E0B4C017
:10159000A0928A01B09289011093520100935101E7
:1015A000F0924E01E0924D01D0935001C0934F0153
:1015B00090924C01D0925401C092530125E09CC0FE
:1015C000A0928A01B09289011093520100935101B7
:1015D000F0924E01E0924D01D0935001C0934F0123
:1015E00090924C01D0925401C092530127E084C0E4
:1015F0000E94BA097C0144C00E949E098C3611F4F5
:10160000BB2403C0AA24BB24B3948091860190918B
:1016100087010196909387018093860112CF0E94E3
:10162000BA09882E982C0DCFA0928A01B092890118
:101630001093520100935101F0924E01E0924D013E
:10164000D0935001C0934F0190924C01D09254011D
:10165000C092530120E0FF24F3944FC00E94BA09C6
:10166000BC0180EC9DE50E944C13CB01EB01E3E053
:10167000CC0FDD1FEA95E1F7880F991FC80FD91F1E
:10168000CE01B7010E944C138B01DBCE0E94BA0938
:101690006C01D7CEA0928A01B092890110935201B9
:1016A00000935101F0924E01E0924D01D093500110
:1016B000C0934F0190924C01D0925401C0925301BB
:1016C000109287011092860178C0A0928A01B09290
:1016D00089011093520100935101F0924E01E09262
:1016E0004D01D0935001C0934F0190924C01D09284
:1016F0005401C092530129E0FF248CE0889EC00170
:101700001124E22EE80E0AC0809186019091870193
:1017100001969093870180938601E3940E949E092D
:101720008B3291F3833281F30CC0809186019091CA
:10173000870101969093870180938601EA940E9425
:101740009E098D3291F3C0915101D0915201815384
:10175000883058F400914F01109150010E94BA094D
:10176000BC01C8010E944C13EB018E010BC080919B
:10177000860190918701019690938701809386015D
:10178000C00FD11F169507950E949E098E3279F3DE
:1017900080918901882339F0CE01969587958093B1
:1017A0008A01C81BD10940915301FF2011F0EE249A
:1017B000EA94BE018E2D0E942609CDB7DEB7ECE07B
:1017C0000C94D21310926F0090938701809386013E
:1017D00081E080938B0110928A010E94E7090895AD
:1017E0000E94E20B089510926F00909387018093FE
:1017F000860110928B0110928A010E94E7090895D8
:101800000E94F30B08951F920F920FB60F921124AE
:101810002F933F934F935F936F937F938F939F93F8
:10182000AF93BF93EF93FF9380918C0190918D01C3
:10183000019790938D0180938C01019611F5809111
:101840008100887F81608093810080E29EE4909394
:1018500089008093880010928B0010928A00229851
:1018600081E080934B0110926F00809186019091EE
:101870008701892B31F080918801882311F40E941F
:10188000E709FF91EF91BF91AF919F918F917F9168
:101890006F915F914F913F912F910F900FBE0F90DD
:1018A0001F901895282F80918E01882391F481E054
:1018B00080938E0184B18D7C84B985B1826385B9B2
:1018C00081E090E06F9364E06A95F1F76F91019782
:1018D000C9F783B18095822308951F93CF93DF9337
:1018E000182F80918E01882391F481E080938E01DE
:1018F00084B18D7C84B985B1826385B981E090E043
:101900006F9364E06A95F1F76F910197C9F7C12F62
:10191000D0E083B190E08C239D23892BD1F38AE022
:1019200090E00E94C01283B190E08C239D23892B0C
:1019300081F383B18123DF91CF911F9108950E949C
:101940006D0C08951F93CF93DF93182F80918E0114
:10195000882391F481E080938E0184B18D7C84B9D9
:1019600085B1826385B981E090E06F9364E06A9508
:10197000F1F76F910197C9F7C12FD0E083B190E0E3
:10198000809590958C239D23892BC1F38AE090E06C
:101990000E94C01283B190E0809590958C239D2386
:1019A000892B61F383B180958123DF91CF911F91C2
:1019B00008950E94A20C08954AB157985A98289AFF
:1019C00021E030E05C9AC9016F9364E06A95F1F719
:1019D0006F910197C9F789B15C98F9016F9364E041
:1019E0006A95F1F76F913197C9F75C9AF9016F9396
:1019F00064E06A95F1F76F913197C9F75C9887FDBC
:101A0000E1CF4AB9089565B190E0AC0141705070E2
:101A1000440F551F9C012670307053E0220F331F76
:101A20005A95E1F7422B6D7C462B45B92BB1887056
:101A3000907034E0880F991F3A95E1F72F77282BA3
:101A40002BB95C9A81E090E0FC016F9364E06A95A9
:101A5000F1F76F913197C9F75C986F9364E06A95DD
:101A6000F1F76F910197C9F708958AB184618AB936
:101A7000209A84E190E00E94C01280E30E94A20DAF
:101A800086E090E00E94C01280E30E94A20D82E0F6
:101A900090E00E94C01280E30E94A20D82E090E0DC
:101AA0000E94C01280E20E94A20D82E090E00E949B
:101AB000C01288E20E94A20D88E00E94A20D81E07F
:101AC0000E94A20D86E00E94A20D8CE00E94A20D51
:101AD000089580919101882329F481E080939101F8
:101AE0000E94350D0895CF92DF92EF92FF920F93EF
:101AF0001F93082F162F0E94690D0E94DC0CC4B0A2
:101B0000D5B0EAB0FBB05A9828988BB1110F110FDD
:101B1000812B8BB984B1826384B9579A802F8295C7
:101B20008F700E94030D802F8F700E94030DFBB8F1
:101B3000EAB8D5B8C4B81F910F91FF90EF90DF902D
:101B4000CF90089560E00E94730D08958CE00E948C
:101B5000A20D08950E94A60D0895813011F48FE022
:101B600001C08EE00E94A20D08950E94AD0D08955F
:101B7000A2E0B0E0EEEBFDE00C94BE1390E8998398
:101B800090EC9A83082F883008F007E0162F611137
:101B900011E0FE01E10FF11D8181800F0E94A20D75
:101BA0000093900110938F012296E4E00C94DA13D5
:101BB0000E94B80D089581E00E94A20DE5E5F1E0D4
:101BC00080E2819391E0ED35F907D9F71092900109
:101BD00010928F0108950E94DB0D08954F925F923D
:101BE0006F927F928F929F92AF92BF92CF92DF922D
:101BF000EF92FF920F93DF93CF93CDB7DEB72A9783
:101C00000FB6F894DEBF0FBECDBF4B015C010AE0FA
:101C10002E010894411C511CC501B4012AE030E09A
:101C200040E050E00E94731369017A0101503201D3
:101C3000600E711CC701B6012AE030E040E050E0C0
:101C40000E942113861A970AA80AB90A882D805D76
:101C5000F3018083C114D104E104F10461F0460171
:101C60005701DACFF701E00FF11D61E080810E949A
:101C7000730D0F5F04C07E010894E11CF11C0A3053
:101C800088F32A960FB6F894DEBF0FBECDBFCF9172
:101C9000DF910F91FF90EF90DF90CF90BF90AF90CA
:101CA0009F908F907F906F905F904F900895EF92EC
:101CB000FF920F931F937B018C0197FF0CC010952F
:101CC0000095F094E094E11CF11C011D111D61E0F0
:101CD0008DE20E94730DC801B7010E94EE0D1F91A5
:101CE0000F91FF90EF9008950E94570E0895CF93A3
:101CF000DF93EC0104C061E00E94730D2196FE01A8
:101D000084918823C1F7DF91CF9108950E94770EC7
:101D10000895CF93DF93EC0104C0219661E00E9407
:101D2000730D88818823C9F7DF91CF9108950E94B0
:101D3000890E089561E00E94730D08950E949A0E25
:101D40000895EF92FF920F931F93CF93DF937C013F
:101D5000062F10E0E3E0000F111FEA95E1F7C0E065
:101D6000D0E09E01200F822F80640E94A20DF70117
:101D7000EC0FFD1FE49161E08E2F0E94730D219600
:101D8000C830D10571F7CDB7DEB7E6E00C94D813B3
:101D90000E94A10E0895519A882311F0599A08952E
:101DA00059980895579A882311F05F9A08955F987B
:101DB0000895882321F480917C008F7D03C0809159
:101DC0007C00806280937C000895EF92FF920F93D5
:101DD0001F9397E890937A0090917C00907F909366
:101DE0007C0090917C008F70892B80937C00809187
:101DF0007A00806480937A00FB01EE24FF2487013F
:101E000080917A00806480937A0080917A0086FDC8
:101E1000FCCF80917C0085FF2BC08091790090E001
:101E2000A0E0B0E0E80EF91E0A1F1B1F319741F732
:101E3000CB01969587956034710538F48E0D9F1D02
:101E400070E00E944C139B010DC0A0E0B0E0E80ED2
:101E5000F91E0A1F1B1F9B0140E050E0C801B7019B
:101E60000E947313C9011F910F91FF90EF90089585
:101E70008091780090917900D3CF64E170E087E0A1
:101E80000E94E50E08950E943D0F08956AE070E0FB
:101E900086E00E94E50EA0E0B0E0BC01CD012CE49C
:101EA0003DE140E050E00E9421132FEF33E040E09D
:101EB00050E00E949513C90108950E94460F0895AD
:101EC000089582E991E00E9454120895462FBC01C2
:101ED00082E991E00E94BA1108950F93DF93CF93A6
:101EE00000D000D00F92CDB7DEB79C01DE01119675
:101EF000EDE5F1E045E001900D924150E1F703E19D
:101F000045E0BE016F5F7F4F82E991E00E940410BF
:101F100082E991E00E94EC0F0E9409130F900F904C
:101F20000F900F900F90CF91DF910F9108950E9425
:101F30006D0F0895FC0111821082138212821582A6
:101F4000148217821682693018F088E0808701C0F9
:101F50006087208B483078F481E090E002C0880FE1
:101F6000991F4A95E2F781878BE290E093878287F9
:101F70008AE290E029C04E3098F4242F30E02850B7
:101F8000304081E090E002C0880F991F2A95E2F767
:101F9000818785E290E09387828784E290E014C095
:101FA0004431A8F4242F30E02E50304081E090E0FE
:101FB00002C0880F991F2A95E2F7818788E290E096
:101FC0009387828787E290E09587848708951586B6
:101FD0001486138612860895DC011C96ED91FC91FF
:101FE0001D97309781F0808119969C911997892BC4
:101FF00080831A96ED91FC911B97908119968C9194
:102000008095892380830895A0E0B0E0EAE0F0E1C4
:102010000C94BA13EC016B01642F7901402F20E07E
:102020000E949A0F19A61AA61BA6FF86EE8630E01C
:1020300041E050E066E2E62EF12C03E210E069E2B6
:1020400070E055C0A32FB0E0F601EA0FFB1F8081BE
:102050008830B8F4FA0102C0EE0FFF1F8A95E2F74C
:10206000CF01FE01EA0FFB1F818B2BA5282B2BA78D
:10207000AA0FBB1FAC0FBD1F5A967C936E93599746
:1020800035C08E30C8F490E00897FA0102C0EE0F18
:10209000FF1F8A95E2F7CF01FE01EA0FFB1F818B3C
:1020A00029A5282B29A7AA0FBB1FAC0FBD1F5A9625
:1020B0001C930E9359971AC08431C0F490E00E9788
:1020C000FA0102C0EE0FFF1F8A95E2F7CF01FE0171
:1020D000EA0FFB1F818B2AA5282B2AA7AA0FBB1F5B
:1020E000AC0FBD1F5A96FC92EE9259973F5F8885C0
:1020F000381708F4A7CFCDB7DEB7E8E00C94D613B5
:10210000A0E0B0E0E6E8F0E10C94B613EC015B016E
:1021100049A5AAA58BA490E009C0E92FF0E0EE0F35
:10212000FF1FEA0DFB1D118210829F5F88859817A3
:10213000A0F384B139A5832B84B987B12AA5822B5A
:1021400087B98AB19BA5892B8AB985B1832B85B9BB
:1021500088B1822B88B98BB1892B8BB9EAE0F0E08A
:102160006F9364E06A95F1F76F913197C9F784B185
:102170003095832384B987B12095822387B98AB1AA
:10218000909589238AB985B1382335B988B1282338
:1021900028B98BB198239BB99090B000C090B10042
:1021A0008091B00083608093B00082E08093B100A2
:1021B000D090B20060E070E03AC05091B2005D197A
:1021C000650F711DE3B0E41609F04FC0F6B0FA16C2
:1021D00009F04BC089B1881509F047C025C0A42F6C
:1021E000B0E09D01220F331F8501020F131FF8017C
:1021F00080819181892BA1F42C0F3D1FF901818DE4
:10220000928DFC01208130E0AC0FBD1F51968C9166
:1022100090E028233923232B19F4F801718360837C
:102220004F5F88854817D8F2D50E4E2DAF2D8E857D
:102230009F856817790708F29092B000C092B100AC
:1022400020E00FC0E22FF0E0EE0FFF1FEA0DFB1DB4
:1022500080819181892B21F48E859F859183808354
:102260002F5F8885281770F305C0E3B0F6B089B0FA
:1022700040E0D7CFCDB7DEB7ECE00C94D213A0E0AE
:10228000B0E0E5E4F1E10C94BA13EC018B01D090DD
:102290007C00E0907A00C7B0F8B080917A0086FDAB
:1022A000FCCF90E009C0E92FF0E0EE0FFF1FE00F38
:1022B000F11F118210829F5F88859817A0F397B154
:1022C0008A8D8095982397B998B1892388B987E832
:1022D00080937A0050E024C0FE01E40FF11D818953
:1022E00080937C0080917A00806480937A00809152
:1022F0007A0086FDFCCFE42FF0E0EE0FFF1FE00F29
:10230000F11F209178003091790080819181820FB6
:10231000931F918380834F5F88854817E8F25F5F42
:10232000898D581710F040E017C040E0F5CFE42F3A
:10233000F0E0EE0FFF1FE00FF11F698D862F90E098
:102340009595879520813181820F931F70E00E94BF
:102350004C13718360834F5F8885481740F3D09298
:102360007C00E0927A00F8B8C7B8CDB7DEB7E8E0F5
:102370000C94D613A0E1B0E0E0ECF1E10C94B913B9
:102380008C017B01D42E842F81508230B0F4D8018F
:102390001C96ED91FC911D97309779F080811996EC
:1023A0009C911997892B80831A96ED91FC911B972C
:1023B000808119969C91892B8083F80180898823DC
:1023C00039F5C02EB12EB701C8010E948010D80186
:1023D0001C96ED91FC911D97309781F080811996A4
:1023E0009C911997892B80831A96ED91FC911B97EC
:1023F000908119968C91809589238083B2E0DB16B9
:1024000009F04EC0BE016F5F7F4F8C2D9B2D22C007
:10241000B701C8010E943F11D8011C96ED91FC91B3
:102420001D97309781F0808119969C911997892B7F
:1024300080831A96ED91FC911B97908119968C914F
:10244000809589238083B2E0DB1651F5BE016F5F72
:102450007F4FC8010E94801040E0BE016F5F7F4F38
:102460001AC0E42FF0E0EE0FFF1F6701CE0EDF1E53
:10247000E60FF71FD8011E962D913C911F97808182
:102480009181281B390BF60180819181820F931F66
:10249000918380834F5FD80118968C91481708F379
:1024A0006096E9E00C94D513CF93DF93EC018A8119
:1024B0009B81009711F00E946B078E819F8100978E
:1024C00011F00E946B0788819981009711F00E949A
:1024D0006B078C819D81009711F00E946B07DF9143
:1024E000CF9108951F920F920FB60F9211242F9340
:1024F0003F934F938F939F93AF93BF932091C201CC
:102500003091C301C90180509C4F9093C3018093C7
:10251000C20180519742C8F08091BE019091BF01E5
:10252000A091C001B091C1010196A11DB11D809380
:10253000BE019093BF01A093C001B093C10120518F
:1025400033423093C3012093C201BF91AF919F9159
:102550008F914F913F912F910F900FBE0F901F9031
:10256000189528EE33E009C0F9016F9364E06A958D
:10257000F1F76F913197C9F701970097A9F708957F
:1025800028EE33E009C0F9016F9364E06A95F1F732
:102590006F913197C9F701970097A9F70895A0E7C0
:1025A000B0E08C918E7F8C93E0EBF0E080818360D3
:1025B0008083E1EBF0E08081807F80838081826096
:1025C0008083B89A8C9181608C93789408958091DF
:1025D000C401882329F481E08093C4010E94CF12B2
:1025E00008950E94E712E0E7F0E080818E7F80830B
:1025F0002091BE013091BF014091C0015091C101B5
:10260000808181608083B901CA0108950E94F1121E
:1026100008950E94E712E0E7F0E080818E7F8083DA
:102620001092BE011092BF011092C0011092C10120
:102630001092C3011092C201B89A80818160808398
:102640000895629FD001739FF001829FE00DF11DFC
:10265000649FE00DF11D929FF00D839FF00D749F1C
:10266000F00D659FF00D9927729FB00DE11DF91FC8
:10267000639FB00DE11DF91FBD01CF011124089525
:10268000991B79E004C0991F961708F0961B881FC4
:102690007A95C9F780950895AA1BBB1B51E107C025
:1026A000AA1FBB1FA617B70710F0A61BB70B881FE2
:1026B000991F5A95A9F780959095BC01CD01089571
:1026C00097FB092E07260AD077FD04D0E5DF06D058
:1026D00000201AF4709561957F4F0895F6F7909554
:1026E00081959F4F0895A1E21A2EAA1BBB1BFD01E5
:1026F0000DC0AA1FBB1FEE1FFF1FA217B307E407E1
:10270000F50720F0A21BB30BE40BF50B661F771F38
:10271000881F991F1A9469F7609570958095909518
:102720009B01AC01BD01CF01089597FB092E052641
:102730000ED057FD04D0D7DF0AD0001C38F45095D6
:102740004095309521953F4F4F4F5F4F0895F6F7D5
:1027500090958095709561957F4F8F4F9F4F08950D
:102760002F923F924F925F926F927F928F929F92A1
:10277000AF92BF92CF92DF92EF92FF920F931F938F
:10278000CF93DF93CDB7DEB7CA1BDB0B0FB6F89440
:10279000DEBF0FBECDBF09942A88398848885F8480
:1027A0006E847D848C849B84AA84B984C884DF80F1
:1027B000EE80FD800C811B81AA81B981CE0FD11DD5
:1027C0000FB6F894DEBF0FBECDBFED010895EE0F3A
:1027D000FF1F0590F491E02D099413E0C2E5D3E0CA
:1027E00004C0FE010E94E9132296C435D107C9F73F
:0427F000F894FFCF8B
:1027F4002020200049522D00202043006333320062
:102804005265642020003E63333200477265656E72
:10281400006D56003E060F067605BD057F0435049F
:10282400D402DD00E5000301EE00F600FD000B011B
:1028340007200000010203030405FF01040400D083
:1028440007F4010F0020202020202020200E0F104C
:0828540011122000C90100006F
:00000001FF
